:020000003428A2
:08000800FF0003088301FE0064
:100010000408FD0079299818181218168C1E0E284D
:100020001A0803142F280C1E1328990003142F28D4
:1000300083178001840AFF3E031D19282F28A3017E
:10004000FC3EA200A309031C2B28FF300000A207DE
:1000500003182628A2070000A30F252808008313F1
:10006000831203130000080083160830990024301F
:100070009800831290309800A00107309F008316EB
:100080008613061386120616851581132030840008
:100090005D3083121920A0308400503019202030A8
:1000A000840030301820061A56285E2886195928F0
:1000B0000A298316861383128617532883168C12F7
:1000C0008312FF30AD00AE01AF01A9010130132052
:1000D0000A301F202D0813200A301F200230132061
:1000E0000A301F202E0813200A301F20033013204F
:1000F0000A301F202F081320AB01AA01AB08031DF3
:10010000B528AB08031D8D282A082D02031C8D2855
:1001100083168613831286179128831686138312FB
:100120008613AB08031D9D282A082E02031C9D2858
:100130008316861283128616A128831686128312CE
:100140008612AB08031DAD282A082F02031CAD2818
:100150008316061383120617B1288316061383121B
:100160000613AA0A0319AB0F7E28AC0A05302C022D
:10017000031D0629A908031DC528AE0A6A212E0AF7
:10018000031DC4280130A900052901302902031DDF
:10019000D128AD036321AD08031DD0280230A9008A
:1001A000052902302902031DDD28AF0A71212F0A1B
:1001B000031DDC280330A900052903302902031D93
:1001C000E928AE036A21AE08031DE8280430A9001F
:1001D000052904302902031DF528AD0A63212D0AE3
:1001E000031DF4280530A900052905302902031D47
:1001F0000029AF037121AF08031DFF28A9010529BC
:10020000FF30AD00AE01AF01A901AC01861909298B
:100210000A297C28C0308B0083168C168312AD010E
:10022000AE01AF01831686128312861283168613DF
:10023000831286138316061383120613AC0106304D
:100240002C0203186229AB01AA01AB08031D5C292B
:10025000AB08031D34292A082D02031C34298316F8
:100260008613831286173829831686138312861302
:10027000AB08031D44292A082E02031C44298316B7
:1002800086128312861648298316861283128612D6
:10029000AB08031D54292A082F02031C5429831676
:1002A00006138312061758298316061383120613A2
:1002B000AA0A0319AB0F2529061A5F295E28AC0A82
:1002C000031D1F291E29013013200A301F202D086D
:1002D00013200800023013200A301F202E0813209C
:1002E0000800033013200A301F202F081320B2010A
:1002F0000800281A7F290B20B200281698290B2005
:10030000B10001303202031D88293108AD00972960
:1003100002303202031D8F293108AE0097290330C5
:100320003202031D96293108AF0097297929281236
:100330007D0884007E088300FF0E7F0E09006300A5
:020340009F29F3
:02400E00623F0F
:00000001FF
